:020000020000FC
:100000000C94910EC7C10000000000000000000029
:1000100000000000000000000000000000000000E0
:10002000000000002DC00000000000009DC0000086
:1000300000000000000000000000000000000000C0
:10004000A6C000000000000000000000000000004A
:100050000000000002030406080C10182030406065
:1000600080000406080C10182030406080A0C000FA
:1000700000070F1F3F0005050D05020503030200E1
:100080004FB662FD0FC0552009F00994C52DC095EB
:10009000089483FDC795C093B200C093410164608A
:1000A0004FBE1895C0910401089483FDC795C09375
:1000B000B200C09341016B7FC0910401CF3F09F4AE
:1000C0001BC04FBE2B982C982D9818952B982C98C8
:1000D0002D9875FD0DC065FD0BC0C5E0CA95F1F703
:1000E000C0915301C0FD2A9AC1FD289AC2FD299AE8
:1000F000209241014FBE18952092B200CC27C160DA
:10010000C7BB6460F5CFC2CF70FFC0CF65FDBECF67
:100110002B9ABCCF70FFBACF65FDB8CF2C9AB6CF63
:1001200070FFB4CF65FDB2CF2D9AB0CF2A9870FF83
:10013000ADCF65FDABCFC1E4CA95F1F72B9AA6CF41
:10014000289870FFA3CF65FDA1CFC1E4CA95F1F750
:100150002C9A9CCF299870FF99CF65FD97CFC1E469
:10016000CA95F1F72D9A92CF4FB6C0916F00CD7F0F
:10017000C0936F006E7FC0918400CE0DD09185003A
:10018000DF1DD0938900C09388004FBE18953FB6FD
:100190008F7EADB3A170A2118061A0E0ADBBA09134
:1001A0006E00AE7FA0936E007894A0910801AA2300
:1001B00041F085FD2BC0A0910801AA95A0930801EC
:1001C00025C040E050E085FD15C0A9B196FDA09581
:1001D000A2FD4FEFA3E096FDA2E0A0936900AA273D
:1001E000A160ACBB8D7FA9B196FDA095A2FD5FEF8C
:1001F000451739F7A8E161FDA093080185FD03C00B
:10020000A8E1A093080140933701816085FD0EC0ED
:10021000A0910901AA2331F0A0910901AA95A09308
:10022000090104C08061AA27A160ACBB80FF38C06F
:10023000A09137014A2F61FF8E7F85FD18C0403F96
:1002400008F040EFA42FA295AF704A0F50915801CB
:10025000533069F0A695A69550FD01C0A69552FDB4
:1002600003C0A41B4A2F03C04A0F08F44FEFA0910C
:1002700040014A1708F44A2F40930101A72FA670A6
:1002800079F0A0910D01A695A69556E0A50F509185
:100290000101A50FA093010118F4AFEFA093010194
:1002A000A0910101A093030140910301A0913C01A1
:1002B0004A1708F04A2F542EA0914201AA2309F4AC
:1002C00022C0542F5A1B10F4A42F50E0BA2E889449
:1002D000AA1FAA2EA0914401A095AA22A50E58F00B
:1002E000A0914301A21509F0AA95AA0EA09343017B
:1002F00048F04A2D08C0A0914301BA1608F0A39512
:10030000A09343014FEF40930401A52DA03408F0C2
:100310006860A0910001A395A093000161F0F8949A
:10032000A0916E00A160A0936E0084FF02C0A1E0C6
:10033000ADBB3FBE1895A0911401A395A0931401E5
:1003400041E050910801552329F085FF03C05A95DB
:1003500050930801A0913701A13018F020923A0182
:100360000DC020923B0120924501A0913A01AF5F60
:10037000A0933A0118F0AFEFA0933A01F894A0913E
:100380006E00A160A0936E0084FF02C0A1E0ADBB2F
:100390003FBE18953FB640918400509185008F7EF6
:1003A000ADB3A170A2118061A0E0ADBBA0916E00C1
:1003B000AE7FA0936E00789481FD25C0A2E096FDEB
:1003C000A3E0A09369008260A9B196FDA095A2FF69
:1003D00005C0409305015093060141C1A3E096FD7D
:1003E000A2E0A0936900AA27A160ACBB8D7F85FF26
:1003F00001C028C140E0A9B196FDA095A2FD22C18F
:100400004093370111C1A3E096FDA2E0A0936900DB
:100410008D7F61FF72C0A2E096FDA3E0A09369000A
:10042000AA27A160ACBB8260409332015093330194
:10043000A09030014A19B09031015B09BB24A22C75
:100440004C38520518F42092360149C0A09176012B
:10045000AA2359F1483C520528F4A0E1BA2EAAE09B
:10046000AA2E23C04836A1E05A0728F4A8E0BA2EE5
:10047000AFE0AA2E1AC0403DA2E05A0728F4A4E03B
:10048000BA2EAEE1AA2E11C0403AA5E05A0728F4D0
:10049000A2E0BA2EACE3AA2E08C04839A8E05A0759
:1004A00020F4A1E0BA2EA8E7AA2EC42EA091340110
:1004B000CA1AD52EA0913501DA0ADD202AF4AFEF51
:1004C000C094D094CA1ADA0A20923601A8E0A21089
:1004D000A0E0CA14DA0618F4A1E0A0933601409314
:1004E00034015093350140913201509133014093D2
:1004F00030015093310102E097C0A09105014A1BE1
:10050000A09106015A0B94FD82C093FD80C092FD1C
:100510007CC086FF03C0D52EC42E0CC056954795CF
:1005200091FD73C05695479590FD6FC0D52EC42E92
:10053000D694C79461FD19C0AC2DAC51AD2DA2402D
:1005400008F005C0DD2089F4AC2DA85C70F4A09102
:100550000701A395AA2311F0A0930701AA3008F47C
:1005600071C02092370181606DC0A0910701AA235C
:1005700019F0AA95A0930701A22C50915C0197FD58
:1005800006C0A0906A01533011F4A0907201AAEF46
:10059000AA0EA22DA21DCA18DA0A4FB74170533015
:1005A00049F4442321F087FD05C0806803C087FF1C
:1005B00001C08F77442359F0533031F4AFEFC0942A
:1005C000D094CA1ADA0A03C040E050E020C0533089
:1005D00049F4CC0CDD1CAAE0CA1AD20818F4A0E039
:1005E000CA2ED22CAFEFCA16D20418F04FEF50E04B
:1005F0000EC0A0914E01CA9E412D000C441F50E038
:1006000008F012C04FEF50E00FC05695479594FF89
:1006100007C0552309F04FEFA42FA6954A0F521D8E
:100620004F3F520508F04FEF40933701816061FF63
:1006300009C0AFE1A095A923AB299A2F8F7DBB20DC
:1006400009F48062A8E1A093080185FF03C0AAE035
:10065000A093080161FD03C085FD01C08F7E85FD6B
:1006600003C0A6E0A0930901F894A0916E00A160D8
:10067000A0936E0084FF02C0A1E0ADBB3FBE189501
:1006800011E00AC013E008C01AE006C01EE104C071
:1006900014E602C018EC00C005E1BB27BA95F1F7DB
:1006A0000A95D9F71A95C1F708952AE338E709C0E2
:1006B00020E33CE806C02AE234EB03C025E238EC34
:1006C00000C012E095FD9F7D95FF9062BB272898A2
:1006D000BA95F1F72C9ABA95F1F72C98BA95F1F7EB
:1006E000289ABA95F1F72B9AB0914F01BA95F1F784
:1006F0002B98B7E8BA95F1F71A9521F7022FB22F88
:10070000BA95F1F70A95D9F73A95D9F62898089548
:10071000221B39E0001F3A9509F40895221F211B7E
:1007200018F4210F8894F6CF0894F4CF622C722C21
:10073000B0E08894B395221F331FE0F737952795D3
:100740008894912E802E020B130B10F4192D082D76
:1007500010F4889401C00894661C771CBA9571F750
:10076000172D062D0895322D11232AF43A95009560
:100770001095031B130BF894029F712C002D129FF0
:10078000912C802C7894780C172D921C292DB4E094
:100790006B2E2695179507956A94D9F7332321F088
:1007A00000951095031B130B0895089510911B01DC
:1007B000169500911A010795B0911F01B01B0B2FE0
:1007C000B0912001B10B1B2F28F40038BFEF1B079D
:1007D00040F009C00F37120508F405C00FE710E01C
:1007E00002C000E81FEF0093240110932501089533
:1007F00000912401B09121010B0F10912501B091BE
:1008000022011B1F20E03091250133230AF42A9591
:10081000B09123012B1F1AF4203F40F00AC02F3063
:1008200008F407C00FEF1FEF2FE003C000E010E057
:1008300020EF30910301B0913C013B1718F43230A6
:1008400030F009C0B0912501BB235AF004C0B0912B
:100850002501BB2332F40093210110932201209340
:10086000230108952091780100912401000F109137
:100870002501111F0E94B30311232AF40038BFEF92
:100880001B0740F009C00F37120508F405C00FE739
:1008900010E002C000E81FEF002352F0B091020107
:1008A000B01B0B2F18F0013008F00AC001E008C09F
:1008B00000950F5FB09102010B0F08F001C00FEF20
:1008C0000093260108952091790100912201109151
:1008D00023010E94B30311232AF40130BFEF1B0749
:1008E00040F009C00F3F120508F405C00FEF10E0FB
:1008F00002C001E01FEF112352F0B0912601B01B9E
:100900000B2F18F0013008F00AC001E008C0009574
:100910000F5FB09126010B0F08F001C00FEF00939D
:10092000030108950FEF677F71FD2AC072FD09C0B2
:100930006860B0911B01BA3020F0B52DB03408F4D6
:10094000677FB0917501BB23D9F0B0911B01BB2328
:10095000B9F00FEF10911B010E948803F894B09139
:10096000130172FDB5E00B9F112D002D789411231A
:1009700009F00FEFB0913F010B1710F400913F0108
:1009800000933E01089500911A0110911B0100543B
:100990001140B0913E0110F4BA9501C0B39511F029
:1009A000B0933E01089500C0089520915701B09181
:1009B0007A00B6FDFACF0091780010917900B091DD
:1009C0007A00BF77B0937A00B0914C01B395B093A1
:1009D0004C01B83060F120924C01B0917401BB23FE
:1009E00021F1112329F0B0914D01BF3F61F009C001
:1009F000B0914D010B1739F020F4BB2321F0BA95CB
:100A000002C0B395E1F300913C01B0934D01B030C9
:100A100050F400ECB03038F400E8B03020F400E4DA
:100A2000B03008F400E000933C01777F0895B09166
:100A30003C01B39511F0B0933C01B0914C01B7303B
:100A400009F47860089502E3F894B0917A010B9F5D
:100A5000012D000C001F7894B0913C010B1710F091
:100A600000913C010093010100930301502E00937B
:100A7000040100933F01089520921A01B0EFB09352
:100A80001B010895F8940091840010918500209135
:100A900014017894309115016090160100931501AE
:100AA00010931601031B160971FD03C076FD81C06A
:100AB0002BC070901701209317012709222311F0F2
:100AC0000FEF1FEF809018019090190130931801DB
:100AD000609219016918161910931C0100911501F3
:100AE000109116010819190920911A0130911B0162
:100AF00036952795020F131F10F40FEF1FEF009389
:100B00001A0110931B0129C020911A0130911B0179
:100B10003901B4E08B2EB2E09B2E343010F08A9471
:100B20009A94383010F08A949A94769467948A94C0
:100B3000E1F726193709992021F0169507959A941F
:100B4000E1F7200F311F20931A0130931B0128F485
:100B50003FEF30931A0130931B01323008F4706478
:100B600071FF02C0B3E00DC0B091660100911101A8
:100B7000023838F0B395003A08F0B395B63008F073
:100B8000B5E09B2EB4E08B2E10911B0100911A0151
:100B900024E0169507952A95E1F70819120928F01F
:100BA000B02FB250B12FB20910F402E010E098015A
:100BB00026C020911A0130911B0139017694679467
:100BC0006694669466942619320906950695200F58
:100BD000321D20931A0130931B01323008F07F7BC5
:100BE00004E0369527953695279526952695201B62
:100BF00010F0223008F422E089019090660160FD37
:100C0000FECFE0902C01F0902D016160B0916F005B
:100C1000B260B0936F00380176FD44C0769467945B
:100C200000932C0110932D01B92DB330E1F0B0FDEC
:100C300004C0060D171D930106C0000F111F0250BE
:100C4000120922E030E0B92DB33068F020932E0174
:100C500030932F01009328011093290160922A01FB
:100C600070922B013DC000932E0110932F01209311
:100C700028013093290160922A0170922B0171FFA3
:100C800010C0B0910D01B33060F000912F011091B0
:100C90001C011595010F28F022F020922E010093DF
:100CA0002F011EC0669400932C01B92DB33091F032
:100CB000B0FD03C0060D262D03C0000F025022E038
:100CC000B92DB33038F020932E01009328016092A3
:100CD0002A0106C000932E012093280160922A0168
:100CE00000911D0102FD0350013039F495FD0EC045
:100CF000B5E0B06CB0937C000DC0023029F4B4E0D4
:100D0000B06CB0937C0006C095FDF2CFB3E0B06C40
:100D1000B0937C0000914401000F10F4BBE60B2758
:100D20000093440160FDFECFB2E0B0930E0161601C
:100D3000B0916F00B260B0936F00B72FB670D1F072
:100D400020911A0130911B0136952795F894009156
:100D5000840010918500020F131F109389000093E7
:100D600088006160B2E0B6BBB0916F00B260B09332
:100D70006F0078940895606120921E0120E067FD65
:100D800020E206C0606120921E0120E267FD20E0A3
:100D9000789401E076FD11C0B72FB67009F06F7E30
:100DA000B0911B01B55048F002E0B55020F003E0CF
:100DB000B55008F006E071FD0AE060FD13C0B09187
:100DC0001E01BB2379F071FF08C0B0910D01B33053
:100DD00020F0B0910E01BA9519F47894706168C052
:100DE0000E949706789400000000F89476FD17C0E2
:100DF00010911B01173008F017E0B5E01B0F72FDD2
:100E000010E183FF110F62FF110F71FD12E8B09125
:100E1000B20060904101B61980F2B10B70F2B0914E
:100E20007B00BF7BB0937B00B0B7B0917B00B06418
:100E3000B0937B00B0911E01B395B0931E01B0B783
:100E400076FD06C0B1E071FDB2E0BA95F1F7B0B73A
:100E5000B072B21709F021C071FF05C003950A30C6
:100E600008F00395AACF64FF93CF6F7E3091840082
:100E70006090850070901A0180901B01370D681CEE
:100E800060928900309388006160B2E0B6BBB09197
:100E90006F00B260B0936F007BCFB0910D01B230A4
:100EA00008F476CF64FD74CF0A9509F086CF7F7E73
:100EB00020912E0130912F01F894B2E0B6BB009141
:100EC000840010918500020F131F10938900009376
:100ED0008800E0902801F09029016160B0916F00D6
:100EE000B260B0936F007894B72FB67039F0B091BC
:100EF0000D0172FFB395B0930D0109C074FF07C0D7
:100F000067FD05C064FD03C0BF91BF917DC5089515
:100F100000E063FF03C064FF01C001E0F89410919A
:100F20001101B7E01B9F212D102D7894200F2695DD
:100F30001795269517952695179510931101183733
:100F400018F4B8E7B093110100911101B0911201AA
:100F50000B1720F060622B982C982D9860FDFECF27
:100F6000E0902A01F0902B016160B0916F00B260B7
:100F7000B0936F000895B2E095FD07C0F894B09368
:100F80001D0128982A9A7894E5C0F894B0931D0121
:100F90002898299A7894DEC0B3E082FF24C095FD9A
:100FA00011C002E0F894B0931D01E0EAF0E0009374
:100FB00053012D98299862FF02C02C9A01C0289AEB
:100FC0007894C8C002E0F894B0931D01E0EAF0E024
:100FD000009353012B982A9862FF02C02C9A01C0FB
:100FE000289A7894B7C095FD0BC0F894B0931D0172
:100FF000EAE8F0E02D9862FF01C02C9A7894AAC02C
:10100000F894B0931D01EAE8F0E02B9862FF01C06C
:101010002C9A78949FC0B4E095FD07C0F894B093E3
:101020001D012A98299A789495C0F894B0931D01CF
:1010300029982A9A78948EC0B5E082FF24C095FD45
:1010400011C001E0F894B0931D01E6E9F0E00093CF
:1010500053012C98289862FF02C02B9A01C02A9A4B
:10106000789478C004E0F894B0931D01EAEAF0E0C7
:10107000009353012C98289862FF02C02D9A01C05A
:10108000299A789467C095FD0BC0F894B0931D0120
:10109000E4E8F0E02C9862FF01C02B9A78945AC0E3
:1010A000F894B0931D01E0E9F0E02C9862FF01C0D4
:1010B0002D9A78944FC0B6E095FD07C0F894B09390
:1010C0001D012998289A789445C0F894B0931D0181
:1010D0002A98289A78943EC0B1E082FF24C095FDFA
:1010E00011C004E0F894B0931D01EAEAF0E0009327
:1010F00053012B982A9862FF02C02D9A01C0299AA9
:10110000789428C001E0F894B0931D01E6E9F0E07E
:10111000009353012D98299862FF02C02B9A01C0B9
:101120002A9A789417C095FD0BC0F894B0931D01CE
:10113000E0E9F0E02B9862FF01C02D9A78940AC094
:10114000F894B0931D01E4E8F0E02D9862FF01C02F
:101150002B9A78946F7D089523E830E0F90120926E
:1011600053012B982C982D982A98289829986B7FB2
:101170000895A4E5B1E00FEF0D930D930D930D933A
:1011800003E00D9304E00D930BE00D9301E00D934C
:1011900001E00D9301E00D93A0E6B1E001E00D93B5
:1011A0000FEF0D930D930D930D930D9303E00D939E
:1011B0000FEF0D930FEF0D930D9305E20D9300EDDF
:1011C0000D930AEF0D930AEF0D9304E00D930FEFCB
:1011D0000D9301E00D9300E00D930AE70D930FEFDF
:1011E0000D9300E00D9301E00D9300E00D9303E0FB
:1011F0000D93089520915B018B7FB0915C01B3301A
:1012000019F09F7DB1FD90629F7BB0915D01B1FDB2
:101210009064223011F0886001C0877F08950A959C
:10122000E00FF21DB4910895E4E5F0E0009154015F
:101230000E940F09B0937801E4E5F0E000915501B8
:101240000E940F09B0937901E2E6F0E000915A01A3
:101250000E940F09B0937A01B09170010FEF1CE06A
:10126000B23011F400EA1AE0B33011F402E815E0EC
:101270000093120110931301E0E7F0E00091770171
:101280000E940F09B09342010895089520916A01C8
:1012900030916B01B0915C01B33009F43E5097FF7F
:1012A00002C020E03FEFB32FB21B6B2EB25810F4F8
:1012B000B2E86B2E00E00395609EB12DBD57D8F3C8
:1012C00000934E01089590680E9446090E944603CB
:1012D00020E030E0B0E16B2E0E944203B091370174
:1012E0002B0F321D6A94C1F7B4E036952795BA9555
:1012F000E1F7822E9F770E9446090895F894E3E073
:10130000F0E0B9E0B7BFB491B078C1F3F894A89514
:10131000B4B7B070B4BFB0916000B861B093600072
:10132000B0E0B0936000B4E0BEBFBFEFBDBF0E94AD
:10133000AC08B0E0B5B9BFE3B4B9B0E0B8B9B0E05B
:10134000B7B9B0E0BBB9B0E0BAB92224A0E0B0E0D0
:101350002D92AA31E9F7A0E0B1E00FEF2D920A95A6
:10136000E9F7B1E0B09344010E94B9080E943F0D33
:10137000B0E0B06CB0937C00B0917A00B460B0681B
:10138000B0937A0000916C0100934F01B1E0B093EB
:101390000A01F8940E944A030E9455030E944603E2
:1013A0000E9458030E9446030E945B030E9446036A
:1013B0000E94D40D0E944A030E944A030E944803DF
:1013C000F8940AEF1AEFA9B196FDA095A2FF1FC0ED
:1013D0001A95C9F70A95B1F7E0E0FCE3B591B43E80
:1013E00039F4B591B03E21F4B591BF3F09F40CC07A
:1013F000E0E0F395F395B591B83F49F4B591B43970
:1014000031F4B591BA3A19F4EE27F69509940E9491
:10141000FA080E9414090E9445090E944609009199
:101420006C0100934F010E94AC08B2E0B5BDB2E080
:10143000B0938100B2E0B093B100B1E0B5BBB0931E
:101440006E00B2E0B6BBB0936F00B1E0B7BBB09333
:101450007000B0917B00BF7BB0937B00B0B7B091C0
:101460007B00B064B0937B000E94400378940E949C
:10147000D304B3E096FDB2E0B0936900B1E0BDBB28
:10148000BB27B160BCBB8D7F0E944A03626033E022
:101490002CE0B0913601BB2321F42CE03A9509F4FD
:1014A0008FCF0E94460380FF8BCF8E7FB091370194
:1014B000B23070F3B92FBF71009139010093380138
:1014C000B0933901B01721F72A9519F76D7FB3E072
:1014D00096FDB2E0B0936900BB27B160BCBB8D7FC5
:1014E000B0917601BB2321F48062B92FB0709B2F9D
:1014F0008F7B209207010E94480385FF05C0B091B1
:101500000701BA3008F080640E94420302E085FFC0
:1015100001C000E0B0913701B017B0F3F8940E9419
:1015200055030E9455030E94550378940E944A0374
:1015300020922701B0915C01B33009F491C00E9460
:101540004203B0916001B13008F48AC0B0910A0141
:10155000B13008F485C085FD1EC0B0913701BF3F92
:1015600008F47EC0F8940E945E0378940E944803B9
:10157000B0913701B130B0F7F8940E9455030E9442
:1015800044030E94550378940E944803B0913701A8
:10159000BF3F90F35EC3B8E09B2E9068F8940E9422
:1015A000460978940E944803F8949F770E94460960
:1015B00080903701B0913701BF37789408F458C054
:1015C0000E944003F8940E945E0378949A9429F74D
:1015D0000E946309B82DB550B0936B010E944A0375
:1015E000F8940E94720D0E94DA0D7894BAE09B2E56
:1015F0009068F8940E94460978940E944803F894F1
:101600009F770E94460980903701B0913701BF371C
:10161000789460F70E944003F8940E9455030E945A
:1016200044030E94550378949A9411F70E94630929
:10163000B82DBB5FB0936A010E944A03F8940E94E0
:10164000720D0E94F70D78940E944803F8940E944E
:1016500046097894B0913701BF3F08F47CCFF9C2B6
:1016600000913701B09127010B1710F0009327016B
:101670000E94480301E0B0915C01B35009F405E019
:10168000B0913701B01708F055CFF8940E945E036F
:101690000E945E030E945E0378940E944A03209297
:1016A0000A0120920B0120920C01B0910B01B3951D
:1016B000B0930B01BF3F79F5B0910C01B395B09396
:1016C0000C01B0916E0109E1BA9559F002E3BA95A7
:1016D00041F00DE7BA9529F00AEFBA9511F0209282
:1016E0000C01B0910C01B017B0F0B0910C01BA959B
:1016F000B0930C01B4EBB0930B01B0916D01B093BA
:101700004F01F8940E945E037894B0916C01B093FD
:101710004F010E9448030E944403B0910801BB237B
:1017200019F485FF01C04CCE01E085FD01C006E043
:10173000B0913701B01708F4B8CFB0915C01B35045
:1017400011F00E944803B0910801BB2309F438CE80
:10175000F8940E94AC08209201012092020120928C
:101760000301522C20920401209243017894B091FD
:101770005901BB0FB093400120921F01209220011C
:1017800020922101209222012092230120924C01DB
:1017900060E070E020921101B8E0B0934C017860F5
:1017A0000E944003B0E073FDB0E0B06CB0937C00E9
:1017B000B0917A00B068B064B0937A00B0917A00CA
:1017C000B6FDFCCF0091780010917900B0917A00BD
:1017D000BF77B0937A00112309F00FEF00934D010A
:1017E0000E94D504B8E0B0934C01786080905B0112
:1017F000B2E0B0935B010E94FA0880925B01F8941A
:10180000BFEFB0933C010E942305B0910101B0935A
:101810003C01B0933D01B0933E017894B1E0B093A8
:101820000101B09303015B2EB0930401B093460114
:10183000B0913B01B0934501B0915C01B33019F414
:101840009F7D87FD90627160726020920D010E9401
:101850005B080E946C080E943C050E9442050E94A1
:101860003C050E9442050E943C0507C0F8940E9476
:10187000FA08789420924C01777F0E94C2060E9459
:10188000D5030E9488070E94BB070E9442050E9460
:10189000BB0666FD0E94D60376FF0E94920476FD89
:1018A0000E94C3040E9488070E94CC070E94420540
:1018B0000E94C20666FD0E94F8030E9488070E94EB
:1018C0000B080E9442050E94BB0666FD0E9432047E
:1018D0000E9488070E941C080E9442050E94C206BE
:1018E00066FD0E9463040E9488070E945B080E94B4
:1018F00042050E94BB06B0E073FDB0E0B06CB0934F
:101900007C00B0917A00B068B064B0937A000E9415
:1019100088070E946C080E9442050E94D50471FF4E
:1019200023C067FD21C0B0913F01B0933C01B0934B
:101930003D01B0913B01B0934501B1E0B093460148
:1019400018E12CE0B0910D01B11740F07D7F74607B
:1019500020930F01BFEFB0933C0106C0B091370157
:10196000B13008F08ACF5AC072FF10C067FD0EC0B8
:10197000B0910F01BA9511F47B7F78CFB0930F012E
:10198000B0913701B13008F078CF48C020921001F3
:10199000B0913A0102E8B01708F040C085FF04C0DA
:1019A000B0910801BB23D1F1B0915C01B33081F457
:1019B00095FD03C087FD04C00BC087FF01C008C0B0
:1019C00067FD06C06068B0913F01B0933C017BCFDA
:1019D00000EF67FF05C0B0913F01B0933C0100E20A
:1019E000B0911B01B01708F448CF67FF17C06F779D
:1019F0009F7D87FD90627460B2E1B0930F01B0915A
:101A00003F01B0933C0139CFB0911001B395B09331
:101A10001001B0913701BB2309F002C020921001E0
:101A2000F8940E94AC0880905B01B2E0B0935B0137
:101A30000E94FA0880925B0120920101209202012B
:101A400020920301522C20920401209240017E7FBB
:101A500078940E9440030E94AC08B0E0B06CB09350
:101A60007C00B0917A00B460B068B0937A0085FFD2
:101A700005C0B0911001B53008F0A2CC12CEEDE057
:101A8000F0E00E946B0D0A3509F01EC0EEE0F0E0B8
:101A90000E946B0D053A09F017C03AE0A4E5B1E0E9
:101AA000E3E0F0E00E946B0D0D9331963A95D1F78B
:101AB00038E1A0E6B1E0EFE0F0E00E946B0D0D939D
:101AC00031963A95D1F704C00E94B9080E94720D70
:101AD000E7E2F0E00895F999FECFE1BDF2BDF89A92
:101AE00000B508950E94950D3AE0A4E5B1E0E3E069
:101AF000F0E00D910E948D0D31963A95D1F738E1C5
:101B0000A0E6B1E0EFE0F0E00D910E948D0D31967E
:101B10003A95D1F70E94A00D0895F999FECF00BD26
:101B2000E1BDF2BDFA9AF99A0895EDE0F0E00FEF09
:101B30000E948D0DEEE0F0E00FEF0E948D0D0895F4
:101B4000EDE0F0E00AE50E948D0DEEE0F0E005EA40
:101B50000E948D0D08953091500100915101313056
:101B600011F400935801323011F4009359013330CD
:101B700011F400935A01343011F4009366013530AA
:101B800011F400935B01363011F400937701373084
:101B900011F400937001383011F400935C01393076
:101BA00011F400935D01089525E00E944A032A95EF
:101BB000E1F708950E9455030E9458030E945B03B9
:101BC0000E945E030E9444030E9455030E94580332
:101BD0000E945B030E945E030E9444030E9455031F
:101BE0000E9458030E945B030E945E0308950E94B6
:101BF0005E030E945B030E9458030E9455030E94EB
:101C000044030E945E030E945B030E9458030E94EB
:101C100055030E9444030E945E030E945B030E94DE
:101C200058030E94550308958090500190905101EF
:101C30000E9455030E9455030E9455030E944403CD
:101C40008A94B1F70E945E030E9444039A94D1F7EC
:101C50000895F8940E94DA0D78940E94D40D0E94A1
:101C6000D40DB1E0B0935001B1E0B0935101209296
:101C70005201F8940E94140E7894B5E06B2E709087
:101C800037010E944A03B09137017B16C1F7B1308A
:101C900018F0BF3F70F10CC00E94AB0DF8940E9489
:101CA000720D0E94DA0DB8E0B09360000E94D40D6E
:101CB0006A9429F7B0915201B395B0935201B330B1
:101CC00008F4D7CF0E94D40DB0915101B395B093D1
:101CD0005101F894B0915001BA95E6E7F0E0EB0FAE
:101CE000F21D049178940395B0915101B01708F456
:101CF000BECF0E94D40D0E94D40DB0915001B39577
:101D0000B0935001B0915001BA3008F4ADCF0E94A9
:101D1000B908F8940E94720DB8E0B09360000E9478
:041D2000D40DECCA28
:00000001FF
